:0600000017C0FECFFDCF8A
:10000600FCCFFBCFFACFDFC0F8CFF7CFF6CFF5CFD7
:10001600AEC0F3CFF2CFF1CFF0CFEFCFEECFEDCF33
:1000260000000100020026000000F894EE27ECBB59
:10003600F1E0FBBFEBBFE5BFF8E1F1BDE1BD8DE04F
:10004600A2E0BB27ED938A95E9F780E094E0A0E66D
:10005600ED930197E9F7E8E2F0E085919591009735
:1000660061F0A591B59105901590BF01F00105903D
:100076000D920197E1F7FB01F0CFEFE5EDBFE4E06C
:10008600EEBFC0E6D1E08AC2E881EFB9779BFECF2A
:10009600EFB16BC01A93B6D2E05C1E2F1A93B6D29C
:1000A600E981B8D218810BC023D3ACD2E05E0E2F03
:1000B6000A93ACD2E0E0AED21E2FE12F1ED32396D8
:1000C6000895C19A979AE8EEF3E0A6D2C198E4E6BD
:1000D600F0E0A2D2C19AE4E6F0E09ED2E6E09AD23F
:1000E600E2E3F0E099D2E1E195D2E2E3F0E094D2E6
:1000F600E1E0EA93E6E993D2E2E0EA93E4ED8FD217
:10010600E3E0EA93ECEF8BD2E4E0EA93E2EE87D207
:10011600E5E087D2E6E085D2E7E083D2E8E081D267
:10012600E9E07FD2EAE07DD2EBE07BD2ECE079D267
:10013600EDE0EA93EFE373D2EEE0EA93EFE36FD2FA
:10014600EFE072D2E0E170D2E1E16ED2E4E16CD28E
:10015600E5E1EA93E0E263D2E6E166D2E7E164D262
:1001660008955D9BFECFE881ECB9219608956A93C8
:100176007A93AA93BA93EA93FA93EFB7EA93A09184
:100186008401B0918501A857BE4FECB1EC93E09184
:100196008401F0918501E857FE4FA081AD3011F43E
:1001A600E1E05E2EA4E8B1E092D2EF5FFF4F6F4F21
:1001B6007F4F97D2E991EFBFF991E991B991A99152
:1001C600799169911895EA93E1E04E2EE991189597
:1001D6001A939798E1E11ED2EAE0F0E01DD2E0E141
:1001E60026D2E2E124D210E0183128F41A935CDF1B
:1001F6001ED21F5FF9CFEDE01AD21991089576D27B
:10020600552079F116D2A03239F4E0918901EA93AA
:10021600E0918A0104D21BC00CD2A03311F4D8DFBE
:1002260016C0A0918901A33411F4D2DF10C0A091A9
:100236008901A43411F4CCDF0AC0FBD1A03411F437
:10024600E89404C0F6D1A03511F4689420F8E0E0F3
:10025600E0938401E0938501E0938601E0938701B2
:10026600552449D224960895E0E0E8BBEEE2E7BBC8
:10027600E0E0E2BBE0E8E1BBE0E0E5BBEFEFE4BBDA
:10028600E8E9EAB9E6E0E0BDE0E0E0BDE8E0E9B9CA
:10029600E5E5EDB9E0E0EEB9EFBDEDE0EEBDE9E094
:1002A600FDE3FBBDEABDE0E1E9BF78940895EF9771
:1002B600E1971A9310E0979AB099FECFE2E1AAD19E
:1002C60011E01C3198F4E12FF0E0DE011196E8D13F
:1002D600EA0FFB1FFF93EF93E0E09CD1AF91BF9134
:1002E600FF2766277727F8D11F5FEBCFED81FE81C9
:1002F6006F817885E1D17F936F93FF93EF93A98503
:10030600BA858B859C8598D1AF91BF918F919F912E
:10031600AAD1AD85BE858F859889A5D1E093600168
:10032600F09361016093620170936301E989FA8930
:100336006B897C89C1D17F936F93FF93EF93AD89CE
:10034600BE898F89988D78D1AF91BF918F919F91FA
:100356008AD1A98DBA8D8B8D9C8D85D1E093640150
:10036600F09365016093660170936701ED8DFE8DD4
:100376006F8D78A1A1D17F936F93FF93EF93A9A17E
:10038600BAA18BA19CA158D1AF91BF918F919F919A
:100396006AD1ADA1BEA18FA198A565D1E0936801F0
:1003A600F093690160936A0170936B01E9A5FAA560
:1003B6006BA57CA581D17F936F93FF93EF93ADA53A
:1003C600BEA58FA598A938D1AF91BF918F919F9166
:1003D6004AD1A9A9BAA98BA99CA945D1E0936C01D8
:1003E600F0936D0160936E0170936F01EDA9FEA904
:1003F6006FA978AD61D17F936F93FF93EF93A9AD0A
:10040600BAAD8BAD9CAD18D1AF91BF918F919F9135
:100416002AD1DE01A35CBF4F0D901D908D919C915A
:10042600D00121D1E0937001F093710160937201C4
:1004360070937301FE01EF5BFF4F01901190619184
:100446007081F00139D17F936F93FF93EF93DE01B3
:10045600AB5BBF4F0D901D908D919C91D001ECD060
:10046600AF91BF918F919F91FED0DE01A75BBF4FE9
:100476000D901D908D919C91D001F5D0E093740163
:10048600F09375016093760170937701FE01E35B4B
:10049600FF4F0190119061917081F0010DD17F9312
:1004A6006F93FF93EF93DE01AF5ABF4F0D901D90F0
:1004B6008D919C91D001C0D0AF91BF918F919F91AA
:1004C600D2D0DE01AB5ABF4F0D901D908D919C91FD
:1004D600D001C9D0E0937801F093790160937A0155
:1004E60070937B01FE01E75AFF4F019011906191D5
:1004F6007081F001E1D07F936F93FF93EF93DE015C
:10050600A35ABF4F0D901D908D919C91D00194D010
:10051600AF91BF918F919F91A6D0DE01AF59BF4F8A
:100526000D901D908D919C91D0019DD0E0937C0102
:10053600F0937D0160937E0170937F01FE01EB597C
:10054600FF4F0190119061917081F001B5D07F93BA
:100556006F93FF93EF93DE01A759BF4F0D901D9048
:100566008D919C91D00168D0AF91BF918F919F9151
:100576007AD0DE01A359BF4F0D901D908D919C91AD
:10058600D00171D0E0938001F093810160938201E4
:10059600709383011881EF96E296089565DE91DDEA
:1005A6002EDE442051F0A0E0A899A1E0E1E0EA2780
:1005B60011F4A89801C0A89A442420FE21C077DE31
:1005C600E0E135D0E1E133D001E010E00930E0E0D0
:1005D6001E07A4F434D069D02AD031D0DF01CB0174
:1005E600E8E052D024D0F801A0E6B1E059D0AE0F31
:1005F600BF1FEC911CD00F5F1F4FE8CFEDE017D067
:10060600CFCFFFCFEA81EF71EA8308953DDDE0E0C9
:10061600EA933ACDEA9338CDFA93EA9318C0EA936F
:1006260039CDEA93E0E6FBCFEA93E0E0F8CFEA9330
:1006360098CDA09188010895E8E01AD00895F801B0
:10064600A0E6B1E02DD0AE0FBF1F3BD00895E991D3
:10065600F991309639F080EA9FE00197F1F7A89575
:100666003197C9F70895EA2BFB2B682B792B089550
:10067600EE230E2EFD01BC0131F0EE0FFF1F661FAB
:10068600771F0A94D1F70895EE230E2EFD01BC01C3
:1006960031F075956795F795E7950A94D1F7089522
:1006A600EE0FFF1FEE0FFF1F0895E62FF72F6627A9
:1006B600F7FD6FEF762F08956E2F7F2FE0E0F0E0C5
:1006C6000895ED91FD916D917C9113970895ED91AB
:1006D600FD916D917D910895ED93FD936D937C93BE
:1006E60008957E936E93FE93EE9308953A932A931C
:1006F6001A930A9308953B812A81198108810895E6
:00000001FF
